******************************************************************************
                  TI ARM Linker PC v18.12.2                    
******************************************************************************
>> Linked Tue Mar 29 14:48:30 2022

OUTPUT FILE NAME:   <app_test.out>
ENTRY POINT SYMBOL: "_c_int00"  address: 00185e0c


MEMORY CONFIGURATION

         name            origin    length      used     unused   attr    fill
----------------------  --------  ---------  --------  --------  ----  --------
  VECTORS               00180000   00000020  00000020  00000000     X
  FLASH0                00180020   0017ffe0  00006acc  00179514  R  X
  FLASH1                00300000   00180000  00000000  00180000  R  X
  STACKS                08000000   00001500  00000000  00001500  RW  
  RAM                   08001500   0003eb00  00000000  0003eb00  RW  


SEGMENT ALLOCATION MAP

run origin  load origin   length   init length attrs members
----------  ----------- ---------- ----------- ----- -------
00180000    00180000    00006aec   00006aec    r-x
  00180000    00180000    00000020   00000020    r-x .intvecs
  00180020    00180020    0000694c   0000694c    r-x .text
  0018696c    0018696c    00000180   00000180    r-- .const


SECTION ALLOCATION MAP

 output                                  attributes/
section   page    origin      length       input sections
--------  ----  ----------  ----------   ----------------
.intvecs   0    00180000    00000020     
                  00180000    00000020     sys_intvecs.obj (.intvecs)

.text      0    00180020    0000694c     
                  00180020    00002cdc     sys_selftest.obj (.text)
                  00182cfc    00000b68     system.obj (.text)
                  00183864    00000898     sys_vim.obj (.text)
                  001840fc    00000664     errata_SSWF021_45.obj (.text)
                  00184760    00000640     pinmux.obj (.text)
                  00184da0    000005bc     esm.obj (.text)
                  0018535c    00000484     gio.obj (.text)
                  001857e0    0000034c     sys_core.obj (.text)
                  00185b2c    000002e0     emif.obj (.text)
                  00185e0c    000002ac     sys_startup.obj (.text:retain)
                  001860b8    00000290     sys_vim.obj (.text:retain)
                  00186348    000001f0     notification.obj (.text)
                  00186538    00000114     esm.obj (.text:retain)
                  0018664c    000000e8     dabort.obj (.text)
                  00186734    000000e0     sys_pmu.obj (.text)
                  00186814    00000068     led.obj (.text)
                  0018687c    00000068     utils.obj (.text)
                  001868e4    00000044     rtsv7R4_T_be_v3D16_eabi.lib : autoinit.c.obj (.text:__TI_auto_init_nobinit_nopinit:__TI_auto_init_nobinit_nopinit)
                  00186928    00000038     sys_main.obj (.text)
                  00186960    00000004     rtsv7R4_T_be_v3D16_eabi.lib : exit.c.obj (.text:abort:abort)
                  00186964    00000004     sys_phantom.obj (.text:retain)
                  00186968    00000004     sys_startup.obj (.text)

.const     0    0018696c    00000180     
                  0018696c    00000180     sys_vim.obj (.const:s_vim_init)

.cinit     0    00180020    00000000     UNINITIALIZED

MODULE SUMMARY

       Module                  code    ro data   rw data
       ------                  ----    -------   -------
    .\drivers\tms_test\source\
       sys_selftest.obj        11484   0         0      
       sys_vim.obj             2856    384       0      
       system.obj              2920    0         0      
       esm.obj                 1744    0         0      
       errata_SSWF021_45.obj   1636    0         0      
       pinmux.obj              1600    0         0      
       gio.obj                 1156    0         0      
       sys_core.obj            844     0         0      
       emif.obj                736     0         0      
       sys_startup.obj         688     0         0      
       notification.obj        496     0         0      
       dabort.obj              232     0         0      
       sys_pmu.obj             224     0         0      
       sys_intvecs.obj         32      0         0      
       sys_phantom.obj         4       0         0      
    +--+-----------------------+-------+---------+---------+
       Total:                  26652   384       0      
                                                        
    .\srcApp\
       sys_main.obj            56      0         0      
    +--+-----------------------+-------+---------+---------+
       Total:                  56      0         0      
                                                        
    .\srcApp\common\
       led.obj                 104     0         0      
       utils.obj               104     0         0      
    +--+-----------------------+-------+---------+---------+
       Total:                  208     0         0      
                                                        
    C:/ti/ccs910/ccs/tools/compiler/ti-cgt-arm_18.12.2.LTS/lib/rtsv7R4_T_be_v3D16_eabi.lib
       autoinit.c.obj          68      0         0      
       exit.c.obj              4       0         0      
    +--+-----------------------+-------+---------+---------+
       Total:                  72      0         0      
                                                        
    +--+-----------------------+-------+---------+---------+
       Grand Total:            26988   384       0      


GLOBAL SYMBOLS: SORTED ALPHABETICALLY BY Name 

address   name                                
-------   ----                                
00186961  C$$EXIT                             
00186954  IntMasterStatusGet                  
UNDEFED   SHT$$INIT_ARRAY$$Base               
UNDEFED   SHT$$INIT_ARRAY$$Limit              
UNDEFED   __TI_CINIT_Base                     
UNDEFED   __TI_CINIT_Limit                    
UNDEFED   __TI_Handler_Table_Base             
UNDEFED   __TI_Handler_Table_Limit            
00185b24  __TI_PINIT_Base                     
00185b28  __TI_PINIT_Limit                    
001868e5  __TI_auto_init_nobinit_nopinit      
ffffffff  __TI_pprof_out_hndl                 
ffffffff  __TI_prof_data_size                 
ffffffff  __TI_prof_data_start                
00180000  __TI_static_base__                  
ffffffff  __binit__                           
ffffffff  __c_args__                          
00185e0c  _c_int00                            
00185a3c  _coreClearAuxiliaryDataFault_       
00185a50  _coreClearAuxiliaryInstructionFault_
00185a14  _coreClearDataFaultAddress_         
001859ec  _coreClearDataFault_                
00185a28  _coreClearInstructionFaultAddress_  
00185a00  _coreClearInstructionFault_         
00185980  _coreDisableEventBusExport_         
001859c4  _coreDisableFlashEcc_               
001859a0  _coreDisableRamEcc_                 
00185970  _coreEnableEventBusExport_          
001859b0  _coreEnableFlashEcc_                
001859d4  _coreEnableIrqVicOffset_            
00185990  _coreEnableRamEcc_                  
00185958  _coreEnableVfp_                     
00185a34  _coreGetAuxiliaryDataFault_         
00185a48  _coreGetAuxiliaryInstructionFault_  
00185a0c  _coreGetDataFaultAddress_           
001859e4  _coreGetDataFault_                  
00185a20  _coreGetInstructionFaultAddress_    
001859f8  _coreGetInstructionFault_           
001857e0  _coreInitRegisters_                 
001858ec  _coreInitStackPointer_              
0018664c  _dabort                             
00185a64  _disable_FIQ_interrupt_             
00185a6c  _disable_IRQ_interrupt_             
00185a5c  _disable_interrupt_                 
00185a74  _enable_interrupt_                  
00185b04  _errata_CORTEXR4_57_                
00185b14  _errata_CORTEXR4_66_                
001840fc  _errata_SSWF021_45_both_plls        
001842f0  _errata_SSWF021_45_pll1             
00184468  _errata_SSWF021_45_pll2             
00185a7c  _esmCcmErrorsClear_                 
00185938  _getCPSRValue_                      
00185940  _gotoCPUIdle_                       
00186790  _pmuDisableCountersGlobal_          
00186780  _pmuEnableCountersGlobal_           
001867ec  _pmuGetCycleCount_                  
001867f4  _pmuGetEventCount_                  
00186800  _pmuGetOverflow_                    
00186734  _pmuInit_                           
001867c0  _pmuResetCounters_                  
001867a0  _pmuResetCycleCounter_              
001867b0  _pmuResetEventCounters_             
001867e0  _pmuSetCountEvent_                  
001867d0  _pmuStartCounters_                  
001867d8  _pmuStopCounters_                   
UNDEFED   _system_post_cinit                  
00186961  abort                               
0018126c  adc1ParityCheck                     
00181358  adc2ParityCheck                     
001863b0  adcNotification                     
ffffffff  binit                               
00181410  can1ParityCheck                     
001814e8  can2ParityCheck                     
001815b0  can3ParityCheck                     
001863c4  canErrorNotification                
001863ec  canMessageNotification              
001863d8  canStatusChangeNotification         
00180030  ccmSelfCheck                        
001826fc  ccmr4GetConfigValue                 
00180938  checkB0RAMECC                       
00180b28  checkB1RAMECC                       
00181c18  checkClockMonitor                   
00180d18  checkFlashECC                       
00181cf4  checkFlashEEPROMECC                 
00181e8c  checkPLL1Slip                       
00181f8c  checkPLL2Slip                       
00182050  checkRAMAddrParity                  
001819d0  checkRAMECC                         
0018215c  checkRAMUERRTest                    
001807bc  checkefcSelfTest                    
00180234  cpuSelfTest                         
00180dfc  cpuSelfTestFail                     
001864f0  crcNotification                     
00183788  customTrimLPO                       
00180df4  custom_dabort                       
00186400  dccNotification                     
0018687c  delayms                             
00182b58  disableParity                       
00186504  dmaGroupANotification               
00180eac  dmaParityCheck                      
001864c8  edgeNotification                    
00180660  efcCheck                            
00182660  efcGetConfigValue                   
00180794  efcSelfTest                         
001806e8  efcStuckZeroTest                    
00186528  emacRxNotification                  
00186518  emacTxNotification                  
00185c14  emifGetConfigValue                  
00185b30  emif_ASYNC1Init                     
00185b7c  emif_ASYNC2Init                     
00185bc8  emif_ASYNC3Init                     
00185b2c  emif_SDRAMInit                      
00185d6c  emif_SDRAM_StartupInit              
00182ad0  enableParity                        
0018276c  errata_PBIST_4                      
00184f24  esmActivateNormalOperation          
00184ff8  esmClearStatus                      
00185038  esmClearStatusBuffer                
00184eec  esmDisableError                     
00184f5c  esmDisableInterrupt                 
00184ec4  esmEnableError                      
00184f34  esmEnableInterrupt                  
00185130  esmEnterSelfTest                    
00184ea8  esmError                            
00185208  esmGetConfigValue                   
00185074  esmGetStatus                        
001850f8  esmGetStatusBuffer                  
00186348  esmGroup1Notification               
00186358  esmGroup2Notification               
00186538  esmHighInterrupt                    
00184da0  esmInit                             
001851b8  esmSelfTestStatus                   
00185054  esmSetCounterPreloadValue           
00184f84  esmSetInterruptLevel                
00184f14  esmTriggerErrorPinReset             
001822c4  fmcBus1ParityCheck                  
0018085c  fmcBus2Check                        
00180898  fmcECCcheck                         
001855bc  gioDisableNotification              
00185554  gioEnableNotification               
001854bc  gioGetBit                           
00185624  gioGetConfigValue                   
001854e4  gioGetPort                          
0018535c  gioInit                             
00186414  gioNotification                     
0018544c  gioSetBit                           
0018542c  gioSetDirection                     
0018549c  gioSetPort                          
001854fc  gioToggleBit                        
00186968  handlePLLLockFail                   
00180f58  het1ParityCheck                     
001810c0  het2ParityCheck                     
001864dc  hetNotification                     
00181004  htu1ParityCheck                     
001811bc  htu2ParityCheck                     
00186428  i2cNotification                     
00186814  initLed                             
0018643c  linNotification                     
00186928  main                                
00182e64  mapClocks                           
00180174  memoryInit                          
00186368  memoryPort0TestFailNotification     
00186384  memoryPort1TestFailNotification     
00181684  mibspi1ParityCheck                  
0018178c  mibspi3ParityCheck                  
001818b0  mibspi5ParityCheck                  
00186464  mibspiGroupNotification             
00186450  mibspiNotification                  
00184760  muxInit                             
001823ec  pbistFail                           
00182470  pbistGetConfigValue                 
001805a8  pbistIsTestCompleted                
001805d4  pbistIsTestPassed                   
00180608  pbistPortTestStatus                 
001804ac  pbistRun                            
001802cc  pbistSelfCheck                      
00180578  pbistStop                           
00182e10  periphInit                          
00186964  phantomInterrupt                    
00184af4  pinmuxGetConfigValue                
001864b0  pwmNotification                     
00180000  resetEntry                          
001863a0  rtiNotification                     
00186478  sciNotification                     
00180020  selftestFailNotification            
00182dd0  setupFlash                          
00182cfc  setupPLL                            
001864a0  spiEndNotification                  
0018648c  spiNotification                     
0018364c  sramGetConfigValue                  
001825bc  stcGetConfigValue                   
001801b8  stcSelfCheck                        
00180df8  stcSelfCheckFail                    
0018308c  systemGetConfigValue                
00182f8c  systemInit                          
0018305c  systemPowerDown                     
001834a0  tcmflashGetConfigValue              
00182d5c  trimLPO                             
00186838  turnOffLed                          
00186828  turnOnLed                           
00186848  turnOverLed                         
00183938  vimChannelMap                       
00183b34  vimDisableInterrupt                 
001839dc  vimEnableInterrupt                  
00183bb8  vimGetConfigValue                   
00183864  vimInit                             
00180e00  vimParityCheck                      
001860b8  vimParityErrorHandler               


GLOBAL SYMBOLS: SORTED BY Symbol Address 

address   name                                
-------   ----                                
00180000  __TI_static_base__                  
00180000  resetEntry                          
00180020  selftestFailNotification            
00180030  ccmSelfCheck                        
00180174  memoryInit                          
001801b8  stcSelfCheck                        
00180234  cpuSelfTest                         
001802cc  pbistSelfCheck                      
001804ac  pbistRun                            
00180578  pbistStop                           
001805a8  pbistIsTestCompleted                
001805d4  pbistIsTestPassed                   
00180608  pbistPortTestStatus                 
00180660  efcCheck                            
001806e8  efcStuckZeroTest                    
00180794  efcSelfTest                         
001807bc  checkefcSelfTest                    
0018085c  fmcBus2Check                        
00180898  fmcECCcheck                         
00180938  checkB0RAMECC                       
00180b28  checkB1RAMECC                       
00180d18  checkFlashECC                       
00180df4  custom_dabort                       
00180df8  stcSelfCheckFail                    
00180dfc  cpuSelfTestFail                     
00180e00  vimParityCheck                      
00180eac  dmaParityCheck                      
00180f58  het1ParityCheck                     
00181004  htu1ParityCheck                     
001810c0  het2ParityCheck                     
001811bc  htu2ParityCheck                     
0018126c  adc1ParityCheck                     
00181358  adc2ParityCheck                     
00181410  can1ParityCheck                     
001814e8  can2ParityCheck                     
001815b0  can3ParityCheck                     
00181684  mibspi1ParityCheck                  
0018178c  mibspi3ParityCheck                  
001818b0  mibspi5ParityCheck                  
001819d0  checkRAMECC                         
00181c18  checkClockMonitor                   
00181cf4  checkFlashEEPROMECC                 
00181e8c  checkPLL1Slip                       
00181f8c  checkPLL2Slip                       
00182050  checkRAMAddrParity                  
0018215c  checkRAMUERRTest                    
001822c4  fmcBus1ParityCheck                  
001823ec  pbistFail                           
00182470  pbistGetConfigValue                 
001825bc  stcGetConfigValue                   
00182660  efcGetConfigValue                   
001826fc  ccmr4GetConfigValue                 
0018276c  errata_PBIST_4                      
00182ad0  enableParity                        
00182b58  disableParity                       
00182cfc  setupPLL                            
00182d5c  trimLPO                             
00182dd0  setupFlash                          
00182e10  periphInit                          
00182e64  mapClocks                           
00182f8c  systemInit                          
0018305c  systemPowerDown                     
0018308c  systemGetConfigValue                
001834a0  tcmflashGetConfigValue              
0018364c  sramGetConfigValue                  
00183788  customTrimLPO                       
00183864  vimInit                             
00183938  vimChannelMap                       
001839dc  vimEnableInterrupt                  
00183b34  vimDisableInterrupt                 
00183bb8  vimGetConfigValue                   
001840fc  _errata_SSWF021_45_both_plls        
001842f0  _errata_SSWF021_45_pll1             
00184468  _errata_SSWF021_45_pll2             
00184760  muxInit                             
00184af4  pinmuxGetConfigValue                
00184da0  esmInit                             
00184ea8  esmError                            
00184ec4  esmEnableError                      
00184eec  esmDisableError                     
00184f14  esmTriggerErrorPinReset             
00184f24  esmActivateNormalOperation          
00184f34  esmEnableInterrupt                  
00184f5c  esmDisableInterrupt                 
00184f84  esmSetInterruptLevel                
00184ff8  esmClearStatus                      
00185038  esmClearStatusBuffer                
00185054  esmSetCounterPreloadValue           
00185074  esmGetStatus                        
001850f8  esmGetStatusBuffer                  
00185130  esmEnterSelfTest                    
001851b8  esmSelfTestStatus                   
00185208  esmGetConfigValue                   
0018535c  gioInit                             
0018542c  gioSetDirection                     
0018544c  gioSetBit                           
0018549c  gioSetPort                          
001854bc  gioGetBit                           
001854e4  gioGetPort                          
001854fc  gioToggleBit                        
00185554  gioEnableNotification               
001855bc  gioDisableNotification              
00185624  gioGetConfigValue                   
001857e0  _coreInitRegisters_                 
001858ec  _coreInitStackPointer_              
00185938  _getCPSRValue_                      
00185940  _gotoCPUIdle_                       
00185958  _coreEnableVfp_                     
00185970  _coreEnableEventBusExport_          
00185980  _coreDisableEventBusExport_         
00185990  _coreEnableRamEcc_                  
001859a0  _coreDisableRamEcc_                 
001859b0  _coreEnableFlashEcc_                
001859c4  _coreDisableFlashEcc_               
001859d4  _coreEnableIrqVicOffset_            
001859e4  _coreGetDataFault_                  
001859ec  _coreClearDataFault_                
001859f8  _coreGetInstructionFault_           
00185a00  _coreClearInstructionFault_         
00185a0c  _coreGetDataFaultAddress_           
00185a14  _coreClearDataFaultAddress_         
00185a20  _coreGetInstructionFaultAddress_    
00185a28  _coreClearInstructionFaultAddress_  
00185a34  _coreGetAuxiliaryDataFault_         
00185a3c  _coreClearAuxiliaryDataFault_       
00185a48  _coreGetAuxiliaryInstructionFault_  
00185a50  _coreClearAuxiliaryInstructionFault_
00185a5c  _disable_interrupt_                 
00185a64  _disable_FIQ_interrupt_             
00185a6c  _disable_IRQ_interrupt_             
00185a74  _enable_interrupt_                  
00185a7c  _esmCcmErrorsClear_                 
00185b04  _errata_CORTEXR4_57_                
00185b14  _errata_CORTEXR4_66_                
00185b24  __TI_PINIT_Base                     
00185b28  __TI_PINIT_Limit                    
00185b2c  emif_SDRAMInit                      
00185b30  emif_ASYNC1Init                     
00185b7c  emif_ASYNC2Init                     
00185bc8  emif_ASYNC3Init                     
00185c14  emifGetConfigValue                  
00185d6c  emif_SDRAM_StartupInit              
00185e0c  _c_int00                            
001860b8  vimParityErrorHandler               
00186348  esmGroup1Notification               
00186358  esmGroup2Notification               
00186368  memoryPort0TestFailNotification     
00186384  memoryPort1TestFailNotification     
001863a0  rtiNotification                     
001863b0  adcNotification                     
001863c4  canErrorNotification                
001863d8  canStatusChangeNotification         
001863ec  canMessageNotification              
00186400  dccNotification                     
00186414  gioNotification                     
00186428  i2cNotification                     
0018643c  linNotification                     
00186450  mibspiNotification                  
00186464  mibspiGroupNotification             
00186478  sciNotification                     
0018648c  spiNotification                     
001864a0  spiEndNotification                  
001864b0  pwmNotification                     
001864c8  edgeNotification                    
001864dc  hetNotification                     
001864f0  crcNotification                     
00186504  dmaGroupANotification               
00186518  emacTxNotification                  
00186528  emacRxNotification                  
00186538  esmHighInterrupt                    
0018664c  _dabort                             
00186734  _pmuInit_                           
00186780  _pmuEnableCountersGlobal_           
00186790  _pmuDisableCountersGlobal_          
001867a0  _pmuResetCycleCounter_              
001867b0  _pmuResetEventCounters_             
001867c0  _pmuResetCounters_                  
001867d0  _pmuStartCounters_                  
001867d8  _pmuStopCounters_                   
001867e0  _pmuSetCountEvent_                  
001867ec  _pmuGetCycleCount_                  
001867f4  _pmuGetEventCount_                  
00186800  _pmuGetOverflow_                    
00186814  initLed                             
00186828  turnOnLed                           
00186838  turnOffLed                          
00186848  turnOverLed                         
0018687c  delayms                             
001868e5  __TI_auto_init_nobinit_nopinit      
00186928  main                                
00186954  IntMasterStatusGet                  
00186961  C$$EXIT                             
00186961  abort                               
00186964  phantomInterrupt                    
00186968  handlePLLLockFail                   
ffffffff  __TI_pprof_out_hndl                 
ffffffff  __TI_prof_data_size                 
ffffffff  __TI_prof_data_start                
ffffffff  __binit__                           
ffffffff  __c_args__                          
ffffffff  binit                               
UNDEFED   SHT$$INIT_ARRAY$$Base               
UNDEFED   SHT$$INIT_ARRAY$$Limit              
UNDEFED   __TI_CINIT_Base                     
UNDEFED   __TI_CINIT_Limit                    
UNDEFED   __TI_Handler_Table_Base             
UNDEFED   __TI_Handler_Table_Limit            
UNDEFED   _system_post_cinit                  

[208 symbols]
